:020000020000FC
:1000000005C06DC018957EC01895189505E007BB12
:1000100000E008BB01E003BF02E009BF03E005BF49
:1000200000E40BBF06B301FBEEF306B301FBEEF7F2
:1000300000E60ABF0DE001BD789403D015D0A89565
:10004000FCCF30FB86F0042D083068F0073258F4FE
:10005000053118F44B7F426006C00B3118F04D7F1C
:10006000446001C0497F0895042F0670002341F4C5
:1000700000E008BB3D7FF8946624772478942EC076
:10008000F894162D272D789441FB9EF4C298326087
:100090000AEF011703E1020710F0C09A0AC0C098E6
:1000A00005EF011707E2020720F4F894662477248D
:1000B000789442FB9EF4C09832600AEF011703E186
:1000C000020710F0C29A0AC0C29805EF011707E2B2
:1000D000020720F4F89466247724789408952FB6C4
:1000E00040FB56F0442450E052BF52E058BF31600C
:1000F00052E055BF416004C03E7F53E055BF4E7F84
:100100002FBE18952FB630FB0EF4439431FB1EF42E
:0A011000639409F473942FBE189550
:00000001FF
